:100000000C9403070C9447070C9447070C9447077C
:100010000C9447070C9447070C9447070C94470728
:100020000C9447070C9447070C9460120C943213FD
:100030000C9447070C9447070C9447070C94470708
:100040000C9447070C940C2C0C9447070C9447070E
:100050000C9447070C9413220C9447070C94470701
:100060000C9447070C9447070C9447070C944707D8
:100070000C9447070C9447070C9447070C944707C8
:100080000C9447070C9447070C9447070C944707B8
:100090000C9447070C9447070C9447070C944707A8
:1000A0000C9447070C9447070C9447079713B91310
:1000B000A414B913A414FB131E14A41473148614EB
:1000C000D417D4170218021844188018801A801AFE
:1000D0009818801A8F198F195A1A801A801A6E1A56
:1000E0000000F0A129002B003900E100E30000002E
:1000F0001E00140004001D0035004D001F001A00F2
:1001000016001B0064004C002000080007000600D9
:1001100050002A0021001500090019004F004A0074
:10012000220017000A0005000000E0002E00015226
:10013000000002520000E200AB0001520000025237
:100140000000E60023001C000B0011000000E4008A
:10015000240018000D00100051004B0025000C0079
:100160000E00360052002C00260012000F0037004F
:1001700031002800270013003300380030004E0003
:100180002D002F003482E500E7000000010001008F
:1001900001000100010000003A001E0231002202AD
:1001A000010001003B001414210235000100010090
:1001B0003C00241425022514010001003D002714F1
:1001C00026022614010001003E0064142E023014A1
:1001D000000001000100010000000100000001001A
:1001E0000100010000000100000001003F0052007A
:1001F00051002302000001004000240021001E00E5
:10020000010001004100250022001F00370001000D
:100210004200260023002000270001004300300296
:1002200030002D14270201004400450001000100A8
:1002300001000000010001000100010001000000B8
:100240003A000100F700FB00010001003B00F40050
:10025000F200FA00FD00F5003C00F000F100F900AA
:10026000FE00F4003D00F500F300FC00FF0001007B
:100270003E000100F800F60000000100010001004E
:100280000000010000000100010001000000010069
:10029000000001003F0001000100B4000000010067
:1002A0004000AA00AC00B600010001004100A80017
:1002B000AD00B5000100B7004200A900AE00B900D2
:1002C0000100B60043000100AB00B70001000100CF
:1002D0004400450001000100010000000A00253033
:1002E000313662003A200025303258000A722F63FE
:1002F0002030313233343536373839414243444582
:10030000460A000A002530325800626F756E636538
:10031000213A20006C6566742073696465206174FD
:100320007461636865640A006C656674207369644F
:1003300065206E6F7420726573706F6E64696E678E
:100340000A00747279696E6720746F207265736534
:1003500074206D637032333031380A000A444542EC
:1003600055473A20656E61626C65642E0A005B73C6
:100370005D004B6579626F617264207374617274A1
:100380002E0A005B575D005B535D005B525D005BB6
:10039000445D005B435D0016034500720067006F1B
:1003A0000044006F007800200045005A000000164D
:1003B000034500720067006F0044006F0078002062
:1003C0000045005A0000000403090409028D0005DD
:1003D0000100A0FA09040000010301010009211134
:1003E000010001223F000705810308000A090401FA
:1003F000000103010200092111010001224D000743
:1004000005820308000A0904020001030000000934
:1004100021110100012236000705830308000A09A3
:100420000403000203000000092111010001222041
:1004300000070584032000010705040320000109CB
:100440000404000103000000092111010001223908
:1004500000070585031000011201100100000008CB
:10046000EDFE071301000102000105010906A101CB
:10047000050719E029E71500250195087501810296
:100480000508190129059505750191029501750366
:100490009101050719002977150025019578750147
:1004A0008102C00631FF0974A1010975150025FFFD
:1004B0009520750881020976150025FF952075089D
:1004C0009102C005010980A101850216010026B72D
:1004D000001A01002AB700751095018100C0050CB3
:1004E0000901A1018503160100269C021A01002AB8
:1004F0009C02751095018100C005010902A1010946
:1005000001A10005091901290515002501950575A9
:100510000181029501750381010501093009311539
:1005200081257F95027508810609381581257F95FB
:100530000175088106050C0A38021581257F950191
:1005400075088106C0C005010906A101050719E06B
:1005500029E71500250195087501810295017508A7
:10056000810105081901290595057501910295017B
:10057000750391010507190029FF150025FF950650
:1005800075088100C00A002530325820006B65795B
:10059000626F6172645F7265706F72743A20000AF4
:1005A0000025303258006B6579626F6172645F7349
:1005B00065745F6C65643A200064656C5F6B657997
:1005C0005F6269743A2063616E27742064656C3AD7
:1005D00020253032580A006164645F6B65795F6280
:1005E00069743A2063616E2774206164643A20253F
:1005F0003032580A00646F6E652E0A00626F6F67B2
:100600006D61676963207363616E3A202E2E2E2020
:1006100000290A002575002F002575005D2800259A
:10062000640020002564002000256400200025646B
:10063000007C0025303258006D6F7573656B6579ED
:10064000205B62746E7C782079207620685D287249
:1006500065702F61636C293A205B006D6B5F776872
:1006600065656C5F74696D655F746F5F6D6178203F
:100670003D2025640A006D6B5F776865656C5F6D72
:1006800061785F7370656564203D2025640A006DA4
:100690006B5F74696D655F746F5F6D6178203D207D
:1006A00025640A006D6B5F6D61785F7370656564CA
:1006B000203D2025640A006D6B5F696E746572765B
:1006C000616C203D2025640A006D6B5F64656C6180
:1006D00079203D2025640A006D6B5F776865656C45
:1006E0005F74696D655F746F5F6D6178203D202573
:1006F000640A006D6B5F776865656C5F6D61785F3C
:100700007370656564203D2025640A006D6B5F741D
:10071000696D655F746F5F6D6178203D2025640AA7
:10072000006D6B5F6D61785F7370656564203D205F
:1007300025640A006D6B5F696E74657276616C206A
:100740003D2025640A006D6B5F64656C6179203D16
:100750002025640A000A00257500363A207768656E
:10076000656C5F74696D655F746F5F6D61783A2069
:10077000000A00257500353A20776865656C5F6D65
:1007800061785F73706565643A20000A0025750022
:10079000343A2074696D655F746F5F6D61783A20DB
:1007A000000A00257500333A206D61785F7370652B
:1007B00065643A20000A00257500323A20696E749B
:1007C000657276616C286D73293A20000A002575E0
:1007D00000313A2064656C6179282A31306D7329C3
:1007E0003A20000A092D2056616C756573202D0A88
:1007F000004D3E004D25643E20003F00736574208F
:1008000064656661756C740A00433E200077686514
:1008100072652064656C74613A20637572736F72DF
:100820003D25642C20776865656C3D25640A536519
:100830006520687474703A2F2F656E2E77696B6926
:1008400070656469612E6F72672F77696B692F4DD0
:100850006F7573655F6B6579730A000A092D204D0A
:100860006F7573656B6579202D0A4553432F713A77
:1008700009717569740A313A0964656C6179282ACD
:1008800031306D73290A323A09696E746572766186
:100890006C286D73290A333A096D61785F7370654E
:1008A00065640A343A0974696D655F746F5F6D61E0
:1008B000780A353A09776865656C5F6D61785F73B2
:1008C000706565640A363A09776865656C5F7469B6
:1008D0006D655F746F5F6D61780A0A703A097072B6
:1008E000696E742076616C7565730A643A09736584
:1008F000742064656661756C74730A75703A092BAF
:10090000310A646F776E3A092D310A706775703A53
:10091000092B31300A7067646F776E3A092D3130D8
:100920000A0A7370656564203D2064656C746120FB
:100930002A206D61785F7370656564202A202872B3
:100940006570656174202F2074696D655F746F5FD9
:100950006D6178290A003F004D3E2000433E200093
:100960004C25640A000A092D20436F6E736F6C6575
:10097000202D0A4553432F713A09717569740A6D28
:100980003A096D6F7573656B65790A000A092D2048
:100990004D61676963202D0A643A09646562756771
:1009A0000A783A096465627567206D6174726978C6
:1009B0000A6B3A096465627567206B6579626F61DD
:1009C00072640A6D3A096465627567206D6F7573AC
:1009D000650A763A0976657273696F6E0A733A0929
:1009E0007374617475730A633A09636F6E736F6C25
:1009F00065206D6F64650A302D343A096C61796544
:100A000072302D34284631302D4634290A50617514
:100A1000733A09626F6F746C6F616465720A653A4C
:100A200009656570726F6D0A6E3A094E4B524F0A36
:100A30007A3A09736C656570204C4544207465737F
:100A4000740A000A002575002E6E6B726F3A200042
:100A50000A002575002E737761705F6261636B73A6
:100A60006C6173685F6261636B73706163653A2088
:100A7000000A002575002E737761705F67726176DA
:100A8000655F6573633A20000A002575002E6E6F5E
:100A90005F6775693A20000A002575002E7377613B
:100AA000705F72616C745F726775693A20000A004A
:100AB0002575002E737761705F6C616C745F6C6775
:100AC00075693A20000A002575002E636170736C09
:100AD0006F636B5F746F5F636F6E74726F6C3A20DD
:100AE000000A002575002E737761705F636F6E7466
:100AF000726F6C5F636170736C6F636B3A20000A96
:100B00000025303258006B65796D61705F636F6EE0
:100B10006669672E7261773A20000A002575002EFB
:100B20006D6F7573653A20000A002575002E6B65A0
:100B300079626F6172643A20000A002575002E6D9B
:100B400061747269783A20000A002575002E656E7E
:100B500061626C653A20000A0025303258006465F5
:100B60006275675F636F6E6669672E7261773A20A0
:100B7000000A0025750064656661756C745F6C61C0
:100B80007965723A20003F004E4B524F3A206F6613
:100B9000660A004E4B524F3A206F6E0A0074696D20
:100BA00065725F636F756E743A202530346C580A35
:100BB000006B6579626F6172645F6E6B726F3A2071
:100BC00025580A006B6579626F6172645F69646CB5
:100BD000653A2025580A006B6579626F6172645F1F
:100BE00070726F746F636F6C3A2025580A00686FDB
:100BF00073745F6B6579626F6172645F6C65647357
:100C000028293A2025580A000A092D2053746174B6
:100C10007573202D0A004743433A20342E382E3274
:100C2000204156522D4C4942433A20312E382E3025
:100C3000204156525F415243483A20617672350A4C
:100C4000004F5054494F4E533A204C554641204294
:100C50004F4F544D41474943204D4F5553454B4508
:100C6000592045585452414B455920434F4E534FFC
:100C70004C4520434F4D4D414E44204E4B524F204A
:100C80003531320A004255494C443A206664616469
:100C90003765632D6469727479202831393A3332AB
:100CA0003A3137204A616E203238203230313629CD
:100CB0000A005649443A2030784645454428457252
:100CC000676F446F7820455A29205049443A2030B4
:100CD0007831333037284572676F446F7820455A32
:100CE00029205645523A203078303030310A0044BD
:100CF0004553433A20742E6D2E6B2E206B6579621E
:100D00006F617264206669726D7761726520666FCB
:100D100072204572676F646F780A000A092D2056A9
:100D2000657273696F6E202D0A000A6D6F757365A9
:100D30003A206F66660A000A6D6F7573653A206F18
:100D40006E0A000A6B6579626F6172643A206F66A1
:100D5000660A000A6B6579626F6172643A206F6E91
:100D60000A000A6D61747269783A206F66660A003B
:100D70000A6D61747269783A206F6E0A000A6465C0
:100D80006275673A206F6E0A000A64656275673A99
:100D9000206F66660A000A0A626F6F746C6F616486
:100DA00065722E2E2E2000433E20006565636F6E17
:100DB0006669673A0A00536C656570204C454420AB
:100DC000746573740A000000000000000000000059
:100DD00000010204060A0F17202C3A4A5D71879D14
:100DE000B3C7DAE9F5FCFFFCF5E9DAC7B39D877113
:100DF0005D4A3A2C20170F0A060402010000000089
:100E000000000000000011241FBECFEFDAE0DEBFBB
:100E1000CDBF04B603FE24C08091F9019091FA0180
:100E2000A091FB01B091FC018730904BA740B04BE3
:100E3000B9F41092F9011092FA011092FB0110928C
:100E4000FC0114BE84B7877F84BF88E10FB6F89495
:100E500080936000109260000FBEE0E0FFE3099510
:100E600011E0A0E0B1E0E4EBFBE502C005900D92DB
:100E7000AA33B107D9F711E0AAE3B1E001C01D928E
:100E8000A93FB107E1F70E949A0F0C94D82D0C945A
:100E90000000FF93EF93E0913A01F0913B0130970E
:100EA00009F00995EF91FF910895FC01859180303B
:100EB00011F0EFDFFBCF0895FF27E0E230E247FFBC
:100EC0000CC0419597FF09C0EDE260957095809543
:100ED0009095611D711D811D911D27FF02C02195F7
:100EE00030E350E2AA27660F771F881F991FAA1FB9
:100EF000A41710F0A41B63955A95A9F7AA3008F01F
:100F0000A95FA05DAF93F39561157105810591050A
:100F100041F7ED3211F4EF93F395F21718F43F9384
:100F2000F395FBCF8F91B5DFFA95E1F70895E9913D
:100F3000F9918591803021F0853219F0AADFF9CF3F
:100F4000089520E0E89455915532C1F3503311F4DF
:100F5000689455915A3348F4505390F3220F022E5F
:100F6000220F220F200D250FF4CF0EF42195899129
:100F70009991533619F3533729F1533559F1BC017F
:100F800088279927E8945C3621F48991999168948F
:100F90005591543639F446EF7EF077FF0DC08FEF50
:100FA0009FEF0AC055374AE039F0583540E121F04B
:100FB000523642E009F00895FF93EF937DDFEF9101
:100FC000FF91B7CFFF93EF93FC0181918030B9F38C
:100FD00060DFFBCFFF93EF9368DFF1CFDF93CF9319
:100FE000CDB7DEB72596A3DFCF91DF9108956111CC
:100FF0000BC0FC018281882321F085EE0E946816D7
:1010000003C085EE0E94301780E090E008950895B7
:101010006091BC017091BD018091BE019091BF01B2
:101020000E94132156985E9825982D9826982E9800
:1010300027982F98813029F0823031F4269A2E9A01
:101040000895259A2D9A089556985E98089588E0F7
:1010500098E0892B11F00E94080880E090E0089544
:1010600056985E9825982D9826982E9827982F9810
:101070008FEF90E0909389008093880090938B008D
:1010800080938A0090938D0080938C00259A2D9AEE
:101090002FEF80E792E0215080409040E1F700C0C0
:1010A0000000269A2E9A2FEF80E792E02150804090
:1010B0009040E1F700C00000279A2F9A2FEF80E7B9
:1010C00092E0215080409040E1F700C00000259858
:1010D0002D982FEF80E792E0215080409040E1F77B
:1010E00000C0000026982E982FEF80E792E0215054
:1010F00080409040E1F700C0000027982F98569854
:101100005E9825982D9826982E9827982F980895C0
:1011100089EA8093800089E08093810024982C984C
:101120003F988AB18F748AB96E98479A8BB1806B59
:101130008BB9769A0E94300887E098E0892B11F0ED
:101140000E94070880E090E0089580E2809300010B
:1011500080913C0181110EC00E94F40881E08093CF
:101160003C012FEF83ED90E3215080409040E1F768
:1011700000C0000080E40E94FA0880930001811101
:101180002EC00E94240980930001811128C00E9472
:10119000240980930001811122C08FE30E94240959
:1011A0008093000181111BC00E941C0980E40E94F1
:1011B000FA0880930001811112C08CE00E9424097A
:1011C0008093000181110BC00E94240980930001CB
:1011D000811105C08FE30E942409809300010E94C1
:1011E0001C098091000108951092B9008AE0809353
:1011F000B800089594EA9093BC009091BC0097FFCA
:10120000FCCF9091B900987F983021F0903111F087
:1012100081E008958093BB0084E88093BC008091B6
:10122000BC0087FFFCCF8091B900887F883111F026
:10123000803471F780E0089584E98093BC00809148
:10124000BC0084FDFCCF08958093BB0084E88093AC
:10125000BC008091BC0087FFFCCF9091B900987FC3
:1012600081E0983209F480E0089584E88093BC001E
:101270008091BC0087FFFCCF8091BB0008958091D6
:101280000001811115C080E40E94FA0880930001DA
:1012900081110CC082E10E94240980930001811118
:1012A00005C08FEF0E942409809300010E941C0951
:1012B00084B1807F84B985B1807F85B98AB1837F0D
:1012C0008AB98BB1837F8BB93E98469808950E9466
:1012D000A508809300010E943F0980B38C7080BBF9
:1012E00081B3836F81BBECE4F1E0AEE3B1E0119236
:1012F0001D9281E0EA35F807D1F788E898E0892B5C
:1013000011F00C94880808959F92AF92BF92CF92EB
:10131000DF92EF92FF920F931F93CF93DF93809111
:1013200000018823E1F080913D018F5F80933D01B2
:10133000811115C082E493E00E9455070E94A50820
:1013400080930001882329F088E293E00E945507EA
:1013500006C084E193E00E9455070E9430080EE326
:1013600011E0C0E0D0E0BB24B39482E0A82ECC24EE
:10137000C394D12C25E0E22E23E0F22EC73000F5F5
:1013800080910001811162C080E40E94FA0880937C
:101390000001811112C082E10E94240980930001A2
:1013A00081110BC0C6010C2E01C0880F0A94EAF708
:1013B00080950E942409809300010E941C0946C068
:1013C000CA30A1F028F4C83059F0C93061F005C026
:1013D000CC3089F070F0CD3089F0209A289810C078
:1013E000219A29980DC0229A2A980AC0239A2B98EC
:1013F00007C0529A01C0539A5B9802C03E9A469821
:10140000E0EAEA95F1F78FB1799985C092E08170B1
:101410008B25892B7C9B02C090E001C094E0892B36
:101420007D9B02C090E001C098E0892B7E9B02C0AA
:1014300090E001C090E1892B9FB19095991F992769
:10144000991F9295990F907E892B10C08091000171
:10145000811176C080E40E94FA08809300018823FD
:1014600009F45BC0912C0E941C09892DF801908120
:10147000981739F1808380910101882301F18091CF
:10148000D70180FF04C08AE093E00E945507809155
:10149000D70180FF0CC0809101011F928F93FF92B2
:1014A000EF920E94EE070F900F900F900F90809197
:1014B000D70180FF04C083E093E00E945507A0920B
:1014C00001010E943F0921960F5F1F4FCE30D105C9
:1014D00009F054CF809101018823B1F081508093AD
:1014E0000101882339F08FE99FE00197F1F700C0EF
:1014F00000000AC0ACE4B1E0EEE3F1E081918D932D
:1015000091E0EC34F907D1F787E298E0892BD1F02C
:101510000E94270817C090E07ACF83E10E94240937
:101520008093000181119ECF81E40E94FA0880938C
:101530000001811197CF0E943509982E909493CF86
:1015400080E094CF81E0DF91CF911F910F91FF90C8
:10155000EF90DF90CF90BF90AF909F900895E82FCD
:10156000F0E0E45BFE4F80810895CF92DF92EF922E
:10157000FF920F931F93CF93DF938CEE92E00E9424
:1015800055073CE4E32E31E0F32EC0E0D0E047EE17
:10159000C42E42E0D42E0EED12E0DF93CF93DF9203
:1015A000CF920E94EE0784EE92E00E945507F70169
:1015B00081917F0190E00E9478219F938F931F93E8
:1015C0000F930E94EE078CED92E00E945507219642
:1015D0008DB79EB708960FB6F8949EBF0FBE8DBF0D
:1015E000CE30D105D1F6DF91CF911F910F91FF90B1
:1015F000EF90DF90CF9008958B3B910578F4883A77
:10160000910540F5853A9105D0F48430910508F0B4
:10161000B1C08130910509F4ADC06BC0803E910529
:1016200008F467C0883E910508F4A4C09C01205FBF
:1016300031092031310508F05CC090650895853A84
:10164000910509F459C0863A910509F458C083E818
:1016500090E40895883A910509F454C0893A9105B7
:1016600009F453C08A3A910509F452C08B3A9105A6
:1016700009F451C08C3A910509F450C08D3A910596
:1016800009F44FC0803B910509F44EC08E3A910594
:1016900009F44DC08F3A910509F44CC0813B910586
:1016A00009F44BC0823B910509F44AC0833B910584
:1016B00009F449C0843B910509F448C0853B910574
:1016C00009F447C0863B910509F446C0873B910564
:1016D00009F445C0883B910509F444C0893B910554
:1016E00009F443C08A3B910509F042C08AE296E4BE
:1016F000089580E090E0089581E890E4089582E8FC
:1017000090E4089582EE94E4089589EE94E40895B7
:101710008AEE94E4089585EB94E4089586EB94E4CE
:10172000089587EB94E408958CEC94E408958DEC8F
:1017300094E4089583E895E408958AE895E408958B
:1017400082E995E4089584E995E4089581E296E4B8
:10175000089583E296E4089584E296E4089585E28C
:1017600096E4089586E296E4089587E296E4089563
:1017700080E094E40895089596E0799FF0011124A3
:1017800094E5899FE00DF11D1124E60FF11DEE0F88
:10179000FF1FEC51FF4F859194910895880F991F79
:1017A000805A9040FC01859194910895880F991F6B
:1017B00080529F4FFC0185919491089526E0729F7D
:1017C000F001112444E5849FE00DF11D1124E60F82
:1017D000F11DEE0FFF1FEC51FF4F25913491C90110
:1017E0009A9581159F4110F4C9010895C90190523D
:1017F0008115904128F4C9019F700E94D60B08956D
:10180000C90190538115904120F4C9019927906C2A
:101810000895211580E5380769F40E94A11A9FEF09
:1018200024E34CE0915020404040E1F700C000002C
:101830000C943822213080E5380751F48CE593E090
:101840000E9455078091D70181608093D701089548
:10185000C90190558115904108F050C0832F9927F8
:101860008F70992781309105D9F4A90143705527CC
:1018700002C0880F991F4A95E2F79C68A90164E0AD
:10188000440F551F6A95E1F744275370842B952B1D
:1018900073E0220F331F7A95E1F7207633271DC0BE
:1018A0008230910529F4922F8827816F906A0895DC
:1018B00083309105A9F4A9014370552781E090E098
:1018C00002C0880F991F4A95E2F79C6843E0220FF7
:1018D000331F4A95E1F7207E3770822B932B0895B2
:1018E0000497F1F4A9014370552781E090E002C00C
:1018F000880F991F4A95E2F79A68E8CFC901905777
:101900008115904120F4C9019F7090620895C9012A
:1019100090588115904120F4C9019F70906A0895F4
:10192000203E3105E0F4203C310558F521333105E6
:1019300009F470C048F42932310509F464C02A3230
:10194000310509F46EC074C029333105F1F0223835
:101950003105D9F02533310509F44EC069C0233E65
:10196000310589F138F4203E3105C1F0223E3105C0
:10197000E1F05EC0263E310569F1273E3105A9F14F
:1019800057C0C9010E94CE0B08958091EA0180FDE5
:1019900002C081FF4DC080EE90E04BC08091EA0113
:1019A00080FFF9CF89E390E044C08091EA0182FF93
:1019B0000EC08091EA0184FF03C080E090E039C04E
:1019C00083EE90E036C08091EA0182FFF2CF82EE92
:1019D00090E02FC08091EA0183FF0BC08091EA0163
:1019E00084FDEBCF87EE90E024C08091EA0183FF75
:1019F000F5CF86EE90E01DC08091EA0185FF07C01B
:101A000089E290E016C08091EA0185FFF9CF85E375
:101A100090E00FC08091EA0186FF07C08AE290E063
:101A200008C08091EA0186FFF9CF81E390E001C010
:101A3000C9010E94FC0A0895089580916D010895DE
:101A40009FB7F89410925C019FBF9091F001943081
:101A500009F058C09091E9009F702091EC0020FFA0
:101A600002C020E801C020E0292B94E09093E90017
:101A70009091EB0090FF43C09091EE0097FF3FC024
:101A800090915A01992321F09091E80095FF37C079
:101A900010925A0196E03091E80035FD15C0309162
:101AA000F001343061F53091EB0035FD28C09150E4
:101AB00021F481E080935A0122C0EFE9FFE03197E1
:101AC000F1F700C00000E7CF8093F1008091E800BB
:101AD00085FD0AC08091E80080FFFCCF8091E8007E
:101AE0008E778093E80006C08FB7F89491E09093CA
:101AF0005C018FBF2F702093E90080E008952F7064
:101B00002093E9008FEF0895CF93DF9300D01F92C9
:101B1000CDB7DEB72091F001243019F523E02983F9
:101B20009B838A832093E9008FEF9091E800815096
:101B300095FD06C095ED9A95F1F700008111F5CF5E
:101B40008091E80085FF0DC040E050E063E070E068
:101B5000CE0101960E9453108091E8008E77809309
:101B6000E8000F900F900F90DF91CF910895CF93E1
:101B7000DF9300D01F92CDB7DEB72091F001243063
:101B800021F522E029839B838A8383E08093E90007
:101B90008FEF9091E800815095FD06C095ED9A95E4
:101BA000F1F700008111F5CF8091E80085FF0DC0AD
:101BB00040E050E063E070E0CE0101960E945310D7
:101BC0008091E8008E778093E8000F900F900F903F
:101BD000DF91CF9108952091F0012430F1F422E0BB
:101BE0002093E9002FEF3091E800215035FD06C029
:101BF00035ED3A95F1F700002111F5CF2091E8007D
:101C000025FF0BC040E050E065E070E00E945310FB
:101C10008091E8008E778093E8000895CF93DF935A
:101C2000EC018091F001843009F047C080910C01F3
:101C30008823E1F080910D018823C1F085E0809335
:101C4000E9008FEF9091E800815095FD06C095E185
:101C50009A95F1F700008111F5CF8091E80085FF9A
:101C60002CC040E050E060E170E017C081E080935C
:101C7000E9008FEF9091E800815095FD06C095ED49
:101C80009A95F1F700008111F5CF8091E80085FF6A
:101C900014C040E050E068E070E0CE010E945310B4
:101CA0008091E8008E778093E80080E1FE01ADE549
:101CB000B1E001900D928A95E1F7DF91CF910895FF
:101CC00083E993E00E9455078091EF01811109C0DB
:101CD0000E94E5110E9442128091E200846080938C
:101CE000E20008958FE893E00E9455071092EF01FB
:101CF00008958BE893E00C94550787E893E00E94E1
:101D000055070C94F92B83E893E00E9455070E9435
:101D1000CF210E94FF2B0E94DE140C941C0D809199
:101D20005B018F5F80935B0162E30E946D2D9111D7
:101D300035C010925B0180915C01882379F180911C
:101D4000F001843049F58091E9008F709091EC00AA
:101D500090FF02C090E801C090E0982B84E080934F
:101D6000E9008091EB0080FF14C08091EE0087FFB6
:101D700010C08091E80085FF03C01092F100F9CFF8
:101D80008091E80080FF05C08091E8008E77809305
:101D9000E8009F709093E90010925C01089542E082
:101DA00061EC81E00E945F1142E061EC82E00E9400
:101DB0005F1142E061EC83E00E945F1142E261EC5E
:101DC00084E00E945F1142E161EC85E00C945F11B8
:101DD0008091F201833009F455C030F4813071F004
:101DE000823009F48EC008958A3009F47AC08B30AD
:101DF00009F460C0893009F09CC020C08091F101D5
:101E0000813A09F096C08091E800877F8093E800CE
:101E10008091F5019091F601892B21F060E080E03E
:101E200090E003C060E18DE591E070E00E949C10BD
:101E30008091E8008B778093E80008958091F1010C
:101E4000813209F076C08091F5019091F6010097FA
:101E500019F0049709F06DC08091E800877F8093A6
:101E6000E8008091E80082FD05C08091F0018111B9
:101E7000F8CF5FC08091F10080936D018091E80000
:101E80008B7753C08091F101813A09F052C0809163
:101E9000F5019091F601892B09F04BC08091E80083
:101EA000877F8093E8008091E80080FFFCCF8091DD
:101EB0000C0136C08091F1018132D9F58091F50194
:101EC0009091F601892BA9F58091E800877F809396
:101ED000E8000E9494118091F30180930C010C940E
:101EE000A11A8091F101813221F58091E800877F6C
:101EF0008093E8000E9494118091F40180936E0118
:101F000008958091F101813AA1F48091E800877FE2
:101F10008093E8008091E80080FFFCCF80916E0103
:101F20008093F1008091E8008E778093E8000C9414
:101F30009411089584B7877F84BF88E10FB6F89421
:101F400080936000109260000FBE90E080E80FB6B2
:101F5000F89480936100909361000FBE0E94671512
:101F60000E94E5110E9442128091E20084608093F9
:101F7000E20080E29DE00E940E2178940E94BC1451
:101F80000E94691582E091E00E94D9140E94E72B1B
:101F900082E793E00E9455078091F001853089F433
:101FA0008EE693E00E9455070E9492218091EE01F7
:101FB000882391F30E94BA21882371F30E943D1077
:101FC000EBCF0E949715E8CF292F33272330310517
:101FD000A9F06CF42130310509F442C022303105FA
:101FE00009F043C08DE890E02BEC33E042C0213291
:101FF0003105C9F02232310519F137C099278130F6
:10200000910541F08230910541F0892B71F5E7ECA3
:10201000F3E005C0EFEAF3E002C0E7E9F3E0849102
:1020200090E09F0126C0653000F5E62FF0E0EE0F4E
:10203000FF1FEB5DFE4F2081318189E090E019C0E8
:10204000653098F4E62FF0E0DF01AA0FBB1FA55E14
:10205000BE4F2D913C91EA5EFE4F808190E009C019
:1020600082E190E028E534E004C080E090E020E0E8
:1020700030E0FA0131832083089580E189BD82E157
:1020800089BD09B400FEFDCF8091D8008F7D80937B
:10209000D8008091E00082608093E0008091E000B1
:1020A00081FDFCCF0895CF92DF92EF92FF920F93C4
:1020B0001F93CF93DF937C018B01EA010E94B5113E
:1020C000811131C0209731F088819981081B190B4B
:1020D000E80EF91EC12CD12C0115110519F18091C2
:1020E000E80085FD14C08091E8008E778093E800B9
:1020F000209741F0888199818C0D9D1D998388835B
:1021000085E011C00E94B511882331F30CC0F7019E
:1021100081917F018093F10001501109FFEFCF1AE7
:10212000DF0ADACF80E0DF91CF911F910F91FF900E
:10213000EF90DF90CF9008952091F7013091F80152
:102140002617370748F06115710539F42091E8002A
:102150002E772093E80001C0B901FC0120E0611551
:102160007105B9F18091F001882309F440C08530F0
:1021700009F43FC08091E80083FD3DC08091E800F4
:1021800082FF06C08091E80082FF26C080E00895AB
:102190008091E80080FFE3CF2091F3008091F2006E
:1021A00090E0922B6115710551F08830910538F45B
:1021B00021912093F100615071090196F3CF21E044
:1021C000089709F020E08091E8008E778093E8007E
:1021D000C6CF2111C7CFD6CF8091F001882339F027
:1021E000853039F08091E80083FFCCCF04C082E0D5
:1021F000089583E0089581E008952091F7013091DA
:10220000F8012617370748F06115710539F4209158
:10221000E8002E772093E80001C0B901FC0120E01E
:1022200061157105C1F18091F001882309F441C065
:10223000853009F440C08091E80083FD3EC0809164
:10224000E80082FF06C08091E80082FF27C080E09E
:1022500008958091E80080FFE3CF2091F300809102
:10226000F20090E0922B6115710559F088309105CC
:1022700040F424912093F100319661507109019648
:10228000F2CF21E0089709F020E08091E8008E77F6
:102290008093E800C5CF2111C6CFD5CF8091F00142
:1022A000882339F0853039F08091E80083FFCBCF67
:1022B00004C082E0089583E0089581E00895982F96
:1022C000973058F59093E900981739F07091EC0029
:1022D0002091ED005091F00003C0242F762F50E0A4
:1022E00021FF19C03091EB003E7F3093EB0030911D
:1022F000ED003D7F3093ED003091EB003160309385
:10230000EB007093EC002093ED005093F0002091CF
:10231000EE0027FF07C09F5FD3CF8F708093E90047
:1023200081E0089580E008958091F10187FD05C066
:102330008091E80080FF0EC012C08091E80082FD0D
:1023400005C08091F0018111F8CF08958091E800D7
:102350008B7708C08091F0018111EACF08958091B8
:10236000E8008E778093E80008958091E4009091D2
:10237000E50045E62091EC0020FF21C02091E80017
:1023800020FD21C02091F001222389F0253089F021
:102390002091EB0025FD0FC02091E4003091E50075
:1023A0002817390739F3415041F0C901E3CF82E0E2
:1023B000089583E0089581E0089584E008952091D0
:1023C000E80022FFDFCF80E008950E9453120E94B0
:1023D0005B12E0EEF0E0808181608083E8EDF0E068
:1023E00080818F77808319BCA7EDB0E08C918E7FC0
:1023F0008C9380818F7E80831092EF0108950F93DC
:102400001F93CF93DF930E9453120E945B12C8ED7B
:10241000D0E088818F7788838881806888838881ED
:102420008F7D888319BC1092F0011092EC011092FC
:10243000EE011092ED0100EE10E0F80180818B7F3B
:10244000808388818160888342E060E080E00E9430
:102450005F11E1EEF0E080818E7F8083E2EEF0E0BC
:10246000808181608083808188608083F8018081A1
:102470008E7F8083888180618883DF91CF911F91D7
:102480000F910895E8EDF0E080818F7E8083E7ED85
:10249000F0E080818160808384E082BF81E080936E
:1024A000EF010C94FF11E8EDF0E080818E7F8083D6
:1024B0001092E20008951092DA001092E10008955F
:1024C0001F920F920FB60F9211242F933F934F93A9
:1024D0005F936F937F938F939F93AF93BF93EF938C
:1024E000FF938091E10082FF0BC08091E20082FFA8
:1024F00007C08091E1008B7F8093E1000E948F0EE6
:102500008091DA0080FF1FC08091D80080FF1BC03F
:102510008091DA008E7F8093DA008091D90080FF6D
:102520000DC080E189BD82E189BD09B400FEFDCF07
:1025300081E08093F0010E94600E05C019BC1092EA
:10254000F0010E94720E8091E10080FF19C080911D
:10255000E20080FF15C08091E2008E7F8093E20050
:102560008091E20080618093E2008091D8008062D7
:102570008093D80019BC85E08093F0010E947D0E05
:102580008091E10084FF30C08091E20084FF2CC084
:1025900080E189BD82E189BD09B400FEFDCF809153
:1025A000D8008F7D8093D8008091E1008F7E80934A
:1025B000E1008091E2008F7E8093E2008091E20052
:1025C00081608093E2008091EC01882311F084E027
:1025D00007C08091E30087FF02C083E001C081E073
:1025E0008093F0010E94830E8091E10083FF29C057
:1025F0008091E20083FF25C08091E100877F809376
:10260000E10082E08093F0011092EC018091E10002
:102610008E7F8093E1008091E2008E7F8093E200C4
:102620008091E20080618093E20042E060E080E01F
:102630000E945F118091F00088608093F0000E94FA
:10264000790EFF91EF91BF91AF919F918F917F9103
:102650006F915F914F913F912F910F900FBE0F900F
:102660001F9018951F920F920FB60F9211242F935F
:102670003F934F935F936F937F938F939F93AF930A
:10268000BF93CF93EF93FF93C091E900CF708091F8
:10269000EC001092E9008091F000877F8093F000B9
:1026A00078940E946E131092E9008091F000886087
:1026B0008093F000C093E900FF91EF91CF91BF911B
:1026C000AF919F918F917F916F915F914F913F91CA
:1026D0002F910F900FBE0F901F9018951F93CF93BF
:1026E000DF93CDB7DEB7AA970FB6F894DEBF0FBE63
:1026F000CDBFE1EFF1E08091F100819321E0E93F6E
:10270000F207C9F70E94E80E8091E80083FF1CC120
:102710002091F1013091F201832F90E08A309105F0
:1027200008F012C1FC01EA5AFF4F0C948D2D20389D
:1027300081F0223809F008C18091F5018F708093F3
:10274000E9008091EB0085FB882780F91092E90071
:1027500006C08091ED019091EE01911182609091FF
:10276000E800977F9093E8008093F1001092F100C9
:10277000C5C0822F8D7F09F0E7C0222319F02230D7
:1027800061F0E2C08091F301813009F0DDC03330A7
:1027900009F080E08093EE0128C08091F30181115F
:1027A00024C02091F5012F7009F4CEC02093E900D8
:1027B0008091EB0080FF19C08091EB00333011F461
:1027C000806211C080618093EB0081E090E0022E76
:1027D00001C0880F0A94EAF78093EA001092EA0099
:1027E0008091EB0088608093EB001092E90080916B
:1027F000E800877F86C02111A7C01091F3011F77E1
:102800008091E3008078812B8093E3008091E80041
:10281000877F8093E8000E9494118091E80080FFF8
:10282000FCCF8091E30080688093E300112311F0D6
:1028300083E001C082E08093F00186C020582230FE
:1028400008F082C08091F3019091F4018C3D23E067
:10285000920779F583E08A838AE289834FB7F894F7
:10286000DE01139620E03EE051E2E32FF0E05093CA
:102870005700E49120FF03C0E295EF703F5FEF70D7
:102880008E2F90E0EA3010F0C79601C0C0968D936D
:102890009D932F5F243149F74FBF8091E800877FD8
:1028A0008093E8006AE270E0CE0101960E949C10DD
:1028B00014C0AE014F5F5F4F6091F5010E94E40FBD
:1028C000009709F441C02091E800277F2093E80099
:1028D000BC0189819A810E94FD108091E8008B776C
:1028E0008093E80031C0203879F58091E800877F37
:1028F0008093E8008091EC018093F1008091E800E2
:102900008E778093E8000E9494111EC021111CC094
:102910009091F3019230C0F48091E800877F80931A
:10292000E8009093EC010E9494118091EC018111D8
:1029300004C08091E30087FF02C084E001C081E011
:102940008093F0010E94CF0E8091E80083FF0AC0BF
:102950008091E800877F8093E8008091EB0080629F
:102960008093EB00AA960FB6F894DEBF0FBECDBFE2
:10297000DF91CF911F910895CF938091F00188232B
:10298000B1F08091E9008F709091EC0090FF02C04F
:1029900090E801C090E0C92FC82B1092E900809107
:1029A000E80083FD0E946E13CF70C093E900CF91C1
:1029B000089590937401809373010895E0917301D9
:1029C000F0917401309721F00190F081E02D09948D
:1029D00080E00895FF920F931F93CF93DF938C01B4
:1029E000E0917301F0917401309799F10280F381C5
:1029F000E02D09958091D70182FF2BC080FF04C094
:102A00008DE895E00E945507E80180E1F82E07E87F
:102A100015E08091D70180FF0BC088811F928F93B2
:102A20001F930F930E94EE070F900F900F900F903F
:102A3000FA942196F110EDCF8091D70180FF09C063
:102A400085E895E0DF91CF911F910F91FF900C9455
:102A50005507DF91CF911F910F91FF900895E0915D
:102A60007301F0917401309721F00480F581E02D1D
:102A70000994089520917101309172018217930792
:102A800071F09093720180937101E0917301F09164
:102A90007401309721F00680F781E02D09940895A4
:102AA00020916F01309170018217930771F090931C
:102AB000700180936F01E0917301F0917401309780
:102AC00021F00084F185E02D0994089508950C9477
:102AD00066150E94D5210E9467090C949B22CF9312
:102AE000C82F8091D70182FF1EC080FF04C086EAF4
:102AF00095E00E9455078091D70180FF0CC01F927E
:102B0000CF9321EA35E03F932F930E94EE070F9079
:102B10000F900F900F908091D70180FF04C08FE934
:102B200095E00E9455078C2FCF910C941C0DCF92ED
:102B3000DF92EF92FF920F931F93CF93DF93CDB766
:102B4000DEB72B970FB6F894DEBF0FBECDBF0E9445
:102B5000840936E7E32E31E0F32E00E010E0C02ECA
:102B6000802F0E94AF0AF701D1907F01D826B1F4DF
:102B70000F5F1F4F0E30110591F78FEF89838A8306
:102B80001B820E94DE218160782F9D838C83498186
:102B90005A816B818D810E943A1641C09091D70174
:102BA00091FF04C08B870E94B50A8B8520E030E03E
:102BB0004D2D50E0922FBA01022E02C075956795F7
:102BC0000A94E2F760FF25C02E83CF82EE24E394BF
:102BD000F12C02C0EE0CFF1C9A95E2F790E08E21DA
:102BE0009F2121E0892B09F420E028870E94DE2123
:102BF0008160782F9A8789874E815F8168858A8571
:102C00000E943A16F801EA58FE4F80818E25808393
:102C100006C02F5F3F4F2630310561F6A9CF0E94D5
:102C20000926109175010E94DE141817A1F00E9468
:102C3000DE14809375012B960FB6F894DEBF0FBE9D
:102C4000CDBFDF91CF911F910F91FF90EF90DF905B
:102C5000CF900C946F152B960FB6F894DEBF0FBE75
:102C6000CDBFDF91CF911F910F91FF90EF90DF903B
:102C7000CF900895CF93DF93CDB7DEB72B970FB6E4
:102C8000F894DEBF0FBECDBF4F83588769877A8720
:102C90008B87DE01119686E0FD0111928A95E9F796
:102CA00085E0FE01379601900D928A95E1F7498102
:102CB0005A816B817C818D819E810E946D1D2B9636
:102CC0000FB6F894DEBF0FBECDBFDF91CF91089550
:102CD000CF93C82F882309F4C1C0823859F40E94C9
:102CE000DE1481FDBBC089E30E940C200E94E82015
:102CF00089E30CC0833879F40E94DE1480FDAEC0F5
:102D000083E50E940C200E94E82083E50E945D205C
:102D1000CF910C94E820843859F40E94DE1482FD8F
:102D20009DC087E40E940C200E94E82087E4EECF3B
:102D30008CEF8C0F813A48F48C2F0E94922A8111DB
:102D40008DC08C2F0E940C20E3CF80E28C0F883046
:102D500048F4C77081E001C0880FCA95EAF70E9465
:102D6000AF20D6CF8BE58C0F833078F4C53A29F0AD
:102D7000C63A31F482E890E005C081E890E002C0F4
:102D800083E890E0CF910C943A1588E58C0F83315D
:102D900008F064C0C83A39F1C93A41F1CA3A49F178
:102DA000CB3A51F1CC3A59F1CD3A61F1C03B69F1DE
:102DB000CE3A71F1CF3A79F1C13B81F1C23B89F151
:102DC000C33B91F1C43B99F1C53BA1F1C63BA9F1CD
:102DD000C73BB1F1C83BB9F1C93BC1F1CA3BC9F529
:102DE0008AE292E038C082EE90E035C089EE90E051
:102DF00032C08AEE90E02FC085EB90E02CC086EBCD
:102E000090E029C087EB90E026C08CEC90E023C0D6
:102E10008DEC90E020C083E891E01DC08AE891E04D
:102E20001AC082E991E017C084E991E014C081E200
:102E300092E011C083E292E00EC084E292E00BC007
:102E400085E292E008C086E292E005C087E292E067
:102E500002C080E090E0CF910C945015CF9108957E
:102E6000882309F44BC0823859F40E94DE1481FF94
:102E700045C089E30E940C200E94E82089E30CC031
:102E8000833871F40E94DE1480FF38C083E50E940D
:102E90000C200E94E82083E50E945D200C94E8202D
:102EA000843859F40E94DE1482FF28C087E40E940F
:102EB0000C200E94E82087E4EFCF9CEF980F913A16
:102EC00058F390E2980F983050F4877091E001C069
:102ED000990F8A95EAF7892F0E94B520DFCF9BE5ED
:102EE000980F933020F480E090E00C943A15885AC3
:102EF000833120F480E090E00C94501508958823ED
:102F000021F00E94AF200C94E8200895882321F03E
:102F10000E94B5200C94E8200895CF92DF92EF92A2
:102F2000FF920F931F93CF93DF93CDB7DEB7289710
:102F30000FB6F894DEBF0FBECDBF8C0185E0F8015F
:102F4000DE01119601900D928A95E1F7F80140811A
:102F50003181F280258122952F7083819481892B84
:102F600031F03F3F31F481E04F3F19F403C081E07D
:102F700001C080E080FDC4C249833A8389819A817F
:102F80002F830E94CA1F9E8388870E94C91F0E94A8
:102F90009C1E4E81E42FE295EF70F0E0E05AFF4F67
:102FA0002F8168850C948D2D842F807F142F1F70A6
:102FB000882311F01295107FFF2059F0112309F496
:102FC00054C2812F68870E94BF200E94E820688534
:102FD0004CC2862F0E943017112309F491C2812F11
:102FE0000E94C52028960FB6F894DEBF0FBECDBF55
:102FF000DF91CF911F910F91FF90EF90DF90CF90D5
:103000000C94E820342F307F842F8F70303211F0F1
:103010008295807F662319F0613019F12BC0FF2063
:10302000B1F0222309F493C1213009F090C1289610
:103030000FB6F894DEBF0FBECDBFDF91CF911F91C9
:103040000F91FF90EF90DF90CF900C94CF20222330
:1030500019F0213009F454C28E830E94D2208E814F
:1030600089C1FF2021F0223008F04AC270C121112D
:1030700047C280C1FF2021F0222309F468C1F5C1B5
:10308000222309F477C105C2242F269526952370A3
:1030900030E02115310521F021303105C9F030C271
:1030A000FF2021F0862F942F937002C080E090E0E3
:1030B00028960FB6F894DEBF0FBECDBFDF91CF913B
:1030C0001F910F91FF90EF90DF90CF900C943A15E5
:1030D000FF2021F0862F942F937002C080E090E0B3
:1030E00028960FB6F894DEBF0FBECDBFDF91CF910B
:1030F0001F910F91FF90EF90DF90CF900C9450159F
:10310000862FFF2019F00E948F2402C00E94F7240E
:1031100028960FB6F894DEBF0FBECDBFDF91CF91DA
:103120001F910F91FF90EF90DF90CF900C947C2532
:10313000842F837009F076C0F110E2C1262F22950A
:1031400026952770220F220F862F8F70C82ED12C24
:10315000E12CF12C022E04C0CC0CDD1CEE1CFF1C5B
:103160000A94D2F764FF10C06FE070E080E090E056
:1031700004C0660F771F881F991F2A95D2F76095A4
:1031800070958095909503C060E070E0CB01242F8E
:10319000269526952370422F50E042305105D1F0FC
:1031A0004330510559F16C297D298E299F294130E1
:1031B000510541F128960FB6F894DEBF0FBECDBF82
:1031C000DF91CF911F910F91FF90EF90DF90CF9003
:1031D0000C94C11E6C297D298E299F2928960FB633
:1031E000F894DEBF0FBECDBFDF91CF911F910F913D
:1031F000FF90EF90DF90CF900C94DB1E0E94C11ED9
:10320000C701B60128960FB6F894DEBF0FBECDBF3A
:10321000DF91CF911F910F91FF90EF90DF90CF90B2
:103220000C94A71EFF2019F0842F817001C0869591
:10323000882309F465C1262F229526952770220F31
:10324000220F862F8F70C82ED12CE12CF12C022E4C
:1032500004C0CC0CDD1CEE1CFF1C0A94D2F764FFEA
:1032600010C06FE070E080E090E004C0660F771F50
:10327000881F991F2A95D2F7609570958095909533
:1032800003C060E070E0CB01242F269526952370C3
:10329000422F50E042305105D1F04330510559F1F1
:1032A0006C297D298E299F294130510541F12896AD
:1032B0000FB6F894DEBF0FBECDBFDF91CF911F9147
:1032C0000F91FF90EF90DF90CF900C94951F6C2999
:1032D0007D298E299F2928960FB6F894DEBF0FBE50
:1032E000CDBFDF91CF911F910F91FF90EF90DF90B5
:1032F000CF900C94AF1F0E94951FC701B60128966E
:103300000FB6F894DEBF0FBECDBFDF91CF911F91F6
:103310000F91FF90EF90DF90CF900C947B1F603F58
:10332000C9F118F4603E50F49BC0623F09F460C0DC
:1033300008F44AC0633F09F46FC092C0162F1F7093
:10334000842F8F71FF2099F00E94141F812F2896DF
:103350000FB6F894DEBF0FBECDBFDF91CF911F91A6
:103360000F91FF90EF90DF90CF900C947F170E9409
:10337000351F812F28960FB6F894DEBF0FBECDBF44
:10338000DF91CF911F910F91FF90EF90DF90CF9041
:103390000C948617FF20A1F02111B2C0842F8F71E9
:1033A00028960FB6F894DEBF0FBECDBFDF91CF9148
:1033B0001F910F91FF90EF90DF90CF900C945A1FC8
:1033C000223008F09DC0EACFFF20A1F0842F8F713A
:1033D00028960FB6F894DEBF0FBECDBFDF91CF9118
:1033E0001F910F91FF90EF90DF90CF900C94141FDE
:1033F000FF2061F3842F8F7128960FB6F894DEBFFB
:103400000FBECDBFDF91CF911F910F91FF90EF9035
:10341000DF90CF900C94351FFF2091F0842F8F7197
:1034200028960FB6F894DEBF0FBECDBFDF91CF91C7
:103430001F910F91FF90EF90DF90CF900C94FF1EA3
:1034400028960FB6F894DEBF0FBECDBFDF91CF91A7
:103450001F910F91FF90EF90DF90CF900C94F51E8D
:10346000FF20A1F0222309F4B1CF862F28960FB6B2
:10347000F894DEBF0FBECDBFDF91CF911F910F91AA
:10348000FF90EF90DF90CF900C946816222309F400
:10349000B1CF862F28960FB6F894DEBF0FBECDBFF2
:1034A000DF91CF911F910F91FF90EF90DF90CF9020
:1034B0000C9430174F70C8010E94F70728960FB67A
:1034C000F894DEBF0FBECDBFDF91CF911F910F915A
:1034D000FF90EF90DF90CF900C941A1E4F70C801B0
:1034E00028960FB6F894DEBF0FBECDBFDF91CF9107
:1034F0001F910F91FF90EF90DF90CF900C94BB0B3A
:1035000028960FB6F894DEBF0FBECDBFDF91CF91E6
:103510001F910F91FF90EF90DF90CF9008950E9440
:10352000CC200E94A1200E94E8200E94AA260E948E
:103530007C2580E090E00E943A1580E090E00C94B9
:1035400050150E94BC200C948F1A0E94CA1F292F6C
:1035500022952F7030E02C3031054CF42A303105A3
:103560006CF4225031092230310590F407C02C3020
:10357000310551F02F30310539F00AC0803E10F08E
:10358000803F31F481E0089593FB882780F9089506
:1035900080E00895CF93DF9300D000D01F92CDB785
:1035A000DEB70F900F900F900F900F90DF91CF919B
:1035B0000895CF93DF9300D000D000D0CDB7DEB711
:1035C00026960FB6F894DEBF0FBECDBFDF91CF9128
:1035D00008951F93CF93DF93C091840116E08091EB
:1035E0008501C81799F0D0E01C9FF0011D9FF00DD8
:1035F0001124EA57FE4F4081518162817381848199
:1036000095810E94D91A2196C770E9CFDF91CF9199
:103610001F9108954091B6015091B7016091B80192
:103620007091B9018091BA019091BB010C94D91AA3
:10363000CF938091BB0182958F7009F05FC080911C
:10364000B801882309F45AC020918401A091850112
:103650006091B6017091B7018091B9019091BA0162
:1036600031E06F3F09F030E0B32FC6E02A1709F4CC
:1036700045C0009721F07F3F21F44B2F03C041E06C
:1036800001C040E030E040FD35C0C29FF001C39F63
:10369000F00D1124EA57FE4F418174132BC0408175
:1036A000641328C04281411125C0438154814817C9
:1036B000590710F441505109481B590B483C51051A
:1036C000C8F48091BB018F7080618093BB0186E05C
:1036D000829FF001839FF00D1124E557FE4F8081FA
:1036E0008F708061808386EB91E00E948D17CF916F
:1036F0000C94E91A2F5F3F4F2770B8CFCF910895F0
:10370000CF92DF92EF92FF920F931F93CF93DF93AD
:10371000CDB7DEB762970FB6F894DEBF0FBECDBF50
:103720008C0185E0F801DE011D9601900D928A95CD
:10373000E1F7D8014C9111965C91119712966C911A
:1037400012971396ED90FC9014977091B601E0914A
:10375000B7012091B9013091BA012115310531F03D
:10376000EF3F31F481E07F3F19F403C081E001C0F5
:1037700080E0B82FB170CB2E80FD6CC1D090B80125
:10378000DD2009F4F5C0F091BB01E216F30638F034
:10379000C701821B930B883C910548F09BC0209584
:1037A00030952E0D3F1D283C310508F093C08F2F1A
:1037B000807F09F052C0E51314C0741312C0D62ED6
:1037C00061110FC0FF70F061F093BB010E940A1BF2
:1037D00086EB91E00E948D178091BB01F8018583F3
:1037E0006CC1EF2831F05F3F31F481E04F3F19F4B5
:1037F00003C081E001C080E080FD03C081E0862736
:1038000001C080E0F82FF170FF2E80FF1CC0809176
:1038100084012091850136E0821709F428C190E0E7
:10382000389FF001399FF00D1124EA57FE4F718146
:10383000571306C07081471303C07281671303C01A
:1038400001968770E9CFD62E662309F436C18091A0
:10385000BB0181608093BB0153C0E51308C07413A2
:1038600006C0611104C0D8011596FC93AEC04D8707
:103870005E878D859E856A8B0E94A51A6A8988233A
:1038800029F1D62E662311F12091BB01822F82955A
:103890008F7090E002970CF460C08091B601909117
:1038A000B70198878F831986FB86EA862C87CE011D
:1038B000079651C0E51731F14D875E878D859E854E
:1038C0006A8B0E94A51A6A8981112EC0C8010E94C4
:1038D0008D17A4C08F2F807F69F77E2DF98AE88A23
:1038E00089890E94CA1A86EB91E00E948D17E6EB47
:1038F000F1E086E0DF011D928A95E9F70E940A1B3C
:10390000D12CDBC07413D8CF6111D6CFD801159656
:10391000FC93C8010E948D17E6EBF1E086E0DF0121
:103920001D928A95E9F7C9C0D62E662379F22091B7
:10393000BB01822F82958F7090E0029774F0809186
:10394000B6019091B7019A8389831B82FD82EC8234
:103950002E83CE0101960E948D1786E0F801A6EB1A
:10396000B1E001900D928A95E1F70E94181B6FC09B
:10397000E216F30628F0C701821B930B9C0104C0DA
:10398000209530952E0D3F1D283C310508F052C082
:10399000D62E662309F49ACFE5132CC074132AC0DF
:1039A0008091BB0180FD1DC0982F92959F70C9F03A
:1039B000D80115968C9315979F3039F09F5F92959B
:1039C000907F8F70892B15968C93C8010E948D175C
:1039D00086E0F801A6EBB1E001900D928A95E1F73F
:1039E00036C086E0F801A6EBB1E001900D928A9511
:1039F000E1F763C04D875E878D859E850E94A51A7D
:103A0000882379F086E0F801A6EBB1E001900D92F1
:103A10008A95E1F70E94181B0E940A1BDD24D394AB
:103A20004CC08091BB0181608093BB01C8010E94A2
:103A30008D1743C07E2DF98AE88A89890E94CA1AA7
:103A4000E6EBF1E086E0DF011D928A95E9F70E943E
:103A50000A1B33C0662309F439CF4D875E878D85F5
:103A60009E850E94A51A882309F430CFCBCF4D87BD
:103A70005E878D859E850E94CA1F292F22952F70F3
:103A800030E0223031052CF49F7041F0811106C0E6
:103A90000CC0243031052CF49F7049F4805E8830CE
:103AA00020F0C8010E948D17CF2CDC2C06C0D80155
:103AB00015969C91907F91F7F8CF8D2D62960FB659
:103AC000F894DEBF0FBECDBFDF91CF911F910F9154
:103AD000FF90EF90DF90CF9008951F93CF93DF93E7
:103AE000CDB7DEB72C970FB6F894DEBF0FBECDBFB3
:103AF0004F83588769877A878B879C87CE01079683
:103B00000E94801B8823C1F02F8138858A859B8580
:103B1000892B31F03F3F11F080E003C02F3FE1F7E8
:103B200081E0811147C04F81588569857A858B85F1
:103B30009C850E94D91A3EC086E0FE013796DE01C0
:103B4000119601900D928A95E1F7FF81E8854A85EB
:103B50005B854115510531F0EF3F31F481E0FF3FC6
:103B600019F403C081E001C080E080FD23C02091F2
:103B7000850130E0C9010196877099276091840121
:103B800070E086179707F1F1F983EA835D834C8330
:103B900096E0929FD001939FB00D1124AA57BE4F7B
:103BA000FE01319601900D929A95E1F7809385017F
:103BB0000E94E91A16E0809184019091850189178D
:103BC00079F1189FC00111248A579E4F0E94801BD3
:103BD000882331F1E09184011E9FF0011124EA57FE
:103BE000FE4F4081518162817381848195810E9461
:103BF000D91A8091840190E001968770992780936B
:103C00008401D9CF0E94A11A1092850110928401DB
:103C1000E6EBF1E086E0DF011D928A95E9F7CACF75
:103C20002C960FB6F894DEBF0FBECDBFDF91CF91BB
:103C30001F910895EF92FF920F931F93CF93DF93FD
:103C40009C01009709F471C0F12CEE24E394E90182
:103C50002196F9018491843740F4843008F056C0ED
:103C6000813081F0823021F160C0853709F449C08C
:103C7000C0F19CE7980F903708F057C08F770E94EB
:103C8000301746C089010E5F1F4FFE01849190E2FC
:103C9000980F983050F48770FE2D01C0FF0F8A9561
:103CA000EAF78F2F0E94BF2015C00E94681614C02B
:103CB00089010E5F1F4FFE01849190E2980F9830AA
:103CC00068F48770FE2D01C0FF0F8A95EAF78F2FE9
:103CD0000E94C5200E94E820E8011AC00E94301707
:103CE000FBCF2E5F3F4FFE01C491CC2341F08FE903
:103CF0009FE00197F1F700C00000C150F6CFE90145
:103D000007C0FE01F490E901229602C00E946816E5
:103D10008F2D882341F0EFE9FFE03197F1F700C0E4
:103D200000008150F6CF9E0192CFDF91CF911F917D
:103D30000F91FF90EF90089508956093C0017093E4
:103D4000C1018093C2019093C3010C948F1A0F9309
:103D50001F930091C0011091C1012091C2013091C7
:103D6000C301062B172B282B392B0093C00110936E
:103D7000C1012093C2013093C3011F910F910C9494
:103D80008F1A0F931F930091C0011091C1012091D0
:103D9000C2013091C301062317232823392300933E
:103DA000C0011093C1012093C2013093C3011F9140
:103DB0000F910C948F1A0F931F930091C0011091D3
:103DC000C1012091C2013091C3010627172728277E
:103DD00039270093C0011093C1012093C201309391
:103DE000C3011F910F910C948F1A1092BC01109275
:103DF000BD011092BE011092BF010C948F1A41E0D8
:103E000050E060E070E004C0440F551F661F771F4C
:103E10008A95D2F74093BC015093BD016093BE01D7
:103E20007093BF010C948F1A41E050E060E070E0A5
:103E300004C0440F551F661F771F8A95D2F78091E3
:103E4000BC019091BD01A091BE01B091BF01842B36
:103E5000952BA62BB72B8093BC019093BD01A0930B
:103E6000BE01B093BF010C948F1A41E050E060E0B6
:103E700070E004C0440F551F661F771F8A95D2F764
:103E800040955095609570958091BC019091BD01D1
:103E9000A091BE01B091BF0184239523A623B7232F
:103EA0008093BC019093BD01A093BE01B093BF016C
:103EB0000C948F1A41E050E060E070E004C0440FC1
:103EC000551F661F771F8A95D2F78091BC0190918C
:103ED000BD01A091BE01B091BF0184279527A627FF
:103EE000B7278093BC019093BD01A093BE01B0930E
:103EF000BF010C948F1A0F931F930091BC01109176
:103F0000BD012091BE013091BF01062B172B282B3C
:103F1000392B0093BC011093BD012093BE01309357
:103F2000BF011F910F910C948F1A0F931F93009153
:103F3000BC011091BD012091BE013091BF0106234B
:103F40001723282339230093BC011093BD0120932C
:103F5000BE013093BF011F910F910C948F1A0F93E4
:103F60001F930091BC011091BD012091BE013091C1
:103F7000BF0106271727282739270093BC01109374
:103F8000BD012093BE013093BF011F910F910C948E
:103F90008F1A0895CF92DF92EF92FF920F931F93A3
:103FA000CF93DF93EC01C090C001D090C101E090AD
:103FB000C201F090C3018091BC019091BD01A0911C
:103FC000BE01B091BF01C82AD92AEA2AFB2A0FE113
:103FD00010E0B701A601002E04C0769567955795AD
:103FE00047950A94D2F740FF07C0BE01802F0E9478
:103FF000DE0B8130910539F40150110950F7BE01F3
:1040000080E00E94DE0BDF91CF911F910F91FF9016
:10401000EF90DF90CF90089590910C01992361F17A
:1040200090910D01992341F1982F9695969596952B
:104030009F3088F4E0910E01F0910F01E90FF11D1E
:10404000877021E030E001C0220F8A95EAF7818174
:10405000822B818308959091D70190FF2DC01F92EC
:104060008F9387ED95E09F938F930E94EE070F90BB
:104070000F900F900F90089540910E0150910F01F5
:1040800020E030E09FEFFA01E20FF31F6281681732
:1040900099F09F3F19F4611101C0922F2F5F3F4F9C
:1040A0002E30310581F79F3F39F0FA01E90FF11DFC
:1040B00097FDFA9582830895089590910C019923B4
:1040C00069F190910D01992349F1982F9695969554
:1040D00096959F3090F4E0910E01F0910F01E90F59
:1040E000F11D877021E030E001C0220F8A95EAF7C8
:1040F000209581812823218308959091D70190FFF5
:104100001FC01F928F9389EB95E09F938F930E941E
:10411000EE070F900F900F900F90089540910E01B1
:1041200050910F0120E030E0FA01E20FF31F92817D
:10413000981301C012822F5F3F4F2E303105A1F737
:10414000089581E090E0E0910E01F0910F01E80FF9
:10415000F91F1082019680319105A9F70895909179
:10416000D601982B9093D601089580959091D60111
:1041700098239093D60108951092D60108959091B6
:10418000D501982B9093D501089580959091D501F4
:1041900098239093D50108951092D50108958093A6
:1041A000C40108951092C401089540910E015091E8
:1041B0000F0120E030E080E0FA01E20FF31F91816F
:1041C00091118F5F2F5F3F4F2F303105A9F7089571
:1041D000E0910E01F0910F018091D6018083E09172
:1041E0000E01F0910F0180819091D501892B808380
:1041F0009091C401992361F0E0910E01F0910F01BB
:104200008081892B80830E94D52081111092C40166
:1042100080910E0190910F010C94EA1490933B0150
:1042200080933A010895CF92DF92EF92FF920F931D
:104230001F936C01EE24FF24C114D104E104F104A6
:1042400021F46B017C0180E001C080E133272F2D38
:104250001E2D0D2D011511052105310519F0885F61
:104260006801790197018601A4E036952795179595
:104270000795AA95D1F7011511052105310519F00A
:104280008C5F6801790197018601F2E036952795E8
:1042900017950795FA95D1F70115110521053105F7
:1042A00019F08E5F68017901B701A60176956795CF
:1042B00057954795452B462B472B09F08F5F1F914C
:1042C0000F91FF90EF90DF90CF9008958295982FF7
:1042D0009C7C96959695837344E0849F900111246D
:1042E000922B892F8A7A86959575990F892B089537
:1042F0001F93CF93DF931F92CDB7DEB799830E94B0
:104300006621182F9981892F0E946621212F30E084
:10431000322F2227A901482BCA010F90DF91CF919C
:104320001F9108958091F001843009F11092D80115
:1043300020E488E190E00FB6F894A895809360009F
:104340000FBE2093600083B7817F846083BF83B7F3
:10435000816083BF7894889583B78E7F83BF88E11F
:104360000FB6F89480936000109260000FBE08951D
:1043700008950895CF930E94B8210E9484090E9455
:10438000B921C0E08C2F0E94AF0A811105C0CF5F18
:10439000CE30C1F780E001C081E0CF9108950E9446
:1043A000A11A0E94DE140C941C0D82E084BD93E0DF
:1043B00095BD9AEF97BD80936E0008952FB7F8943E
:1043C0008091D9019091DA01A091DB01B091DC01DB
:1043D0002FBF0895CF92DF92EF92FF920F931F931A
:1043E0002FB7F8944091D9015091DA016091DB0127
:1043F0007091DC012FBF6A017B01EE24FF248C0148
:1044000020E030E0C016D106E206F30610F4415079
:104410005109481B590BCA011F910F91FF90EF9052
:10442000DF90CF9008951F920F920FB60F92112434
:104430008F939F93AF93BF938091D9019091DA01AD
:10444000A091DB01B091DC010196A11DB11D80930B
:10445000D9019093DA01A093DB01B093DC01BF9105
:10446000AF919F918F910F900FBE0F901F90189555
:104470000E94E511F8942FEF87EA91E621508040E1
:104480009040E1F700C0000087E090EBDC018093F2
:10449000F9019093FA01A093FB01B093FC012CE089
:1044A00088E190E00FB6F894A895809360000FBE65
:1044B00020936000FFCFEF92FF920F931F93CF9353
:1044C000DF93E82EF12C8F2D0E94AF0AC0E0D0E0E0
:1044D000082F10E098010C2E02C0359527950A94FC
:1044E000E2F720FD05C02196C630D10599F709C035
:1044F0006C2F7F2D80E00E94BC0BE812F4CF81E08E
:1045000005C0F3948EE0F812DECF80E0DF91CF910A
:104510001F910F91FF90EF900895CF93C82F8CE2D9
:104520000E945B22882321F08C2FCF910C945B2278
:1045300080E0CF910895CF930E94E823811102C0BB
:104540000E94CE238CEF95E00E945507C5E6C1502E
:1045500049F00E9484098FE39CE90197F1F700C0BC
:104560000000F5CF85EF95E00E94550789E20E9493
:104570008D22811111C18AE20E948D2281110E9437
:10458000CE2385E00E948D2281110E9438220E9454
:10459000F3238093D70187E00E948D22882399F12D
:1045A0008BE10E948D22882351F09091D70191FBDD
:1045B000882780F921E0822780FB91F922C08EE0D4
:1045C0000E948D22882351F09091D70192FB882779
:1045D00080F921E0822780FB92F913C080E10E94DC
:1045E0008D229091D701882341F093FB882780F991
:1045F00021E0822780FB93F904C0892F809580FBFE
:1046000090F99093D7018091D7010E94F7230E94DF
:1046100005248093EA0180EE0E948D22882341F0D8
:104620008091EA01982F909590FB80F98093EA01A0
:1046300089E30E948D22882359F09091EA0191FB31
:10464000882780F921E0822780FB91F99093EA0185
:1046500082EE0E948D22882359F09091EA0192FB0C
:10466000882780F921E0822780FB92F99093EA0164
:1046700086EE0E948D22882359F09091EA0193FBE7
:10468000882780F921E0822780FB93F99093EA0143
:1046900083EE0E948D22882359F09091EA0194FBC9
:1046A000882780F921E0822780FB94F99093EA0122
:1046B00085E30E948D22882359F09091EA0195FBB1
:1046C000882780F921E0822780FB95F99093EA0101
:1046D00081E30E948D22882359F09091EA0196FB94
:1046E000882780F921E0822780FB96F99093EA01E0
:1046F00081E10E948D22882359F09091EA0197FB75
:10470000882780F921E0822780FB97F99093EA01BE
:104710008091EA010E9409248091EA0187FB8827A1
:1047200080F980930D0187E20E948D22C82F8EE1CF
:104730000E948D228111C2608FE10E948D22811121
:10474000C46080E20E948D228111C86081E20E94D3
:104750008D228111C06182E20E948D228111C0628E
:1047600083E20E948D228111C06484E20E948D2226
:10477000882311F0C06802C0CC2329F08C2F0E943E
:1047800000246C2F03C00E94FC23682F70E080E09F
:1047900090E0CF910C949D1ECF9108956DEE7EEF29
:1047A00080E090E00E94C32D60E082E090E00E94F3
:1047B000B52D60E083E090E00E94B52D60E084E0DC
:1047C00090E00E94B52D60E085E090E00C94B52D5E
:1047D00080E090E00E94AF2D21E08D3E9E4F09F0D9
:1047E00020E0822F089582E090E00C94A72D682F9E
:1047F00082E090E00C94B52D83E090E00C94A72D1E
:10480000682F83E090E00C94B52D84E090E00C9448
:10481000A72D682F84E090E00C94B52D8091DF01E6
:1048200080FF0BC06091130185E0689FB0011124E7
:1048300075956795759567952AC081FF09C0609148
:10484000130185E0689FB0011124759567951FC01D
:1048500082FF07C06091130185E0689FB0011124B9
:1048600016C04091E0014423C9F06091120146173F
:1048700088F72091130185E0289F90011124429F21
:10488000C001439F900D112470E00E94792D603883
:10489000710540F46115710539F002C065E070E002
:1048A000862F08958FE7089581E008958091DF01B4
:1048B00080FF08C06091110170E07595679575954E
:1048C000679521C081FF06C06091110170E0759568
:1048D000679519C082FF04C06091110170E010C09B
:1048E0008091E0018823C1F0609110018617A0F744
:1048F00090911101989FC001112470E00E94792DC0
:104900006038710528F46115710521F0862F08952E
:104910008FE7089581E0089561E070E0F4CF803F73
:1049200021F40E940E24819504C0813F29F40E9445
:104930000E248093E3010895823F21F40E940E2407
:10494000819504C0833F29F40E940E248093E201E4
:104950000895893F19F40E94562405C08A3F31F416
:104960000E94562481958093E40108958B3F21F4A1
:104970000E945624819504C08C3F29F40E9456243D
:104980008093E5010895843F21F48091E1018160E5
:1049900017C0853F21F48091E101826011C0863FFC
:1049A00021F48091E10184600BC0873F21F4809164
:1049B000E101886005C0883F31F48091E1018061A8
:1049C0008093E10108958D3F21F48091DF018160A2
:1049D0000BC08E3F21F48091DF01826005C08F3FC4
:1049E00029F48091DF0184608093DF010895803F86
:1049F00039F48091E30187FF6CC01092E30169C034
:104A0000813F29F48091E3011816BCF362C09091B4
:104A1000E201823F29F497FF5CC01092E20159C085
:104A2000833F19F41916CCF354C0893F41F48091A7
:104A3000E40118160CF04DC01092E4014AC08A3F00
:104A400029F48091E40187FF44C0F6CF8B3F39F40D
:104A50008091E50187FF3DC01092E5013AC08C3F8F
:104A600029F48091E5011816BCF333C0843F21F48A
:104A70008091E1018E7F17C0853F21F48091E10193
:104A80008D7F11C0863F21F48091E1018B7F0BC0A7
:104A9000873F21F48091E101877F05C0883F31F491
:104AA0008091E1018F7E8093E10113C08D3F21F45D
:104AB0008091DF018E7F0BC08E3F21F48091DF015A
:104AC0008D7F05C08F3F29F48091DF018B7F80931C
:104AD000DF018091E20181110EC08091E30181111B
:104AE0000AC08091E401811106C08091E501811125
:104AF00002C01092E00108958091D70183FF7EC02B
:104B000088E396E00E9455078091E1011F928F9300
:104B100083E396E09F938F930E94EE0781E396E0F4
:104B20000E9455072091E201822F992787FD9095D9
:104B30009F932F938EE296E09F938F930E94EE07B0
:104B40008CE296E00E9455072091E301822F99277D
:104B500087FD90959F932F9389E296E09F938F9383
:104B60000E94EE0787E296E00E9455072091E4013B
:104B7000822F992787FD90959F932F9384E296E04B
:104B80009F938F930E94EE0782E296E00E94550762
:104B90002091E501822F992787FD90959F932F9370
:104BA0008FE196E09F938F930E94EE078CE196E051
:104BB0000E9455078091E0011F928F9389E196E052
:104BC0009F938F930E94EE0787E196E00E9455071E
:104BD0008091DF011F928F9384E196E09F938F93E2
:104BE0000E94EE0781E196E00E9455078DB79EB7BF
:104BF0004C960FB6F8949EBF0FBE8DBF81EE91E02C
:104C00000E942F150E94DE219093DE018093DD012A
:104C100008951F93CF93DF938091DD019091DE0182
:104C20000E94EA214091E001442321F020911401E7
:104C300030E006C0209115015AE0259F9001112413
:104C40008217930708F482C08091E2011091E3017A
:104C5000D091E401C091E501811107C0111105C097
:104C6000D11103C0CC2309F471C04F3F19F04F5F3D
:104C70004093E001181624F40E940E248093E20170
:104C80008091E20187FF05C00E940E2481958093E8
:104C9000E201111624F40E940E248093E301809116
:104CA000E30187FF05C00E940E2481958093E301F4
:104CB0006091E201662339F11091E301112319F1AA
:104CC000772767FD7095872F972F0E947E2C23E30F
:104CD00033E343E35FE30E94E22C0E944B2C60939A
:104CE000E201612F772767FD7095872F972F0E942C
:104CF0007E2C23E333E343E35FE30E94E22C0E9434
:104D00004B2C6093E3011D1624F40E9456248093DB
:104D1000E4018091E40187FF05C00E94562481953B
:104D20008093E4011C1624F40E9456248093E5012C
:104D30008091E50187FF05C00E94562481958093EC
:104D4000E501DF91CF911F910C947C25DF91CF91EC
:104D50001F910895E1EEF1E085E0DF011D928A9553
:104D6000E9F71092E0011092DF0108958BE598E0D9
:104D70000E9455071F9281E08F931F9285E08F93C9
:104D80008DE098E09F938F930E94EE070F900F9015
:104D90000F900F900F900F9008958330E9F128F451
:104DA000813061F0823009F10895853009F462C0E4
:104DB00008F449C0863009F474C0089520911501A3
:104DC000862F90E0820F911D8F3F910520F4620F96
:104DD0006093150103C08FEF809315018091150139
:104DE0001F928F9386E497E072C020911401862F62
:104DF00090E0820F911D8F3F910520F4620F609328
:104E0000140103C08FEF80931401809114011F924D
:104E10008F9384E397E05BC020911301862F90E08D
:104E2000820F911D8F3F910520F4620F6093130153
:104E300003C08FEF80931301809113011F928F9312
:104E400081E297E044C020911201862F90E0820F0A
:104E5000911D8F3F910520F4620F6093120103C0F2
:104E60008FEF80931201809112011F928F938CE03B
:104E700097E02DC020911101862F90E0820F911DA7
:104E80008F3F910520F4620F6093110103C08FEFF3
:104E900080931101809111011F928F9383EF96E00F
:104EA00016C020911001862F90E0820F911D8F3F38
:104EB000910520F4620F6093100103C08FEF80937F
:104EC0001001809110011F928F9388ED96E09F93BF
:104ED0008F930E94EE070F900F900F900F90089500
:104EE000833081F128F4813059F08230D1F0089577
:104EF000853009F449C0B8F1863009F456C00895E8
:104F000080911501681720F4861B8093150102C05B
:104F100010921501809115011F928F9389EC96E0F4
:104F200054C080911401681720F4861B80931401EB
:104F300002C010921401809114011F928F9387EB8D
:104F400096E043C080911301681720F4861B80937C
:104F5000130102C010921301809113011F928F93CD
:104F600084EA96E032C080911201681720F4861B13
:104F70008093120102C010921201809112011F92BF
:104F80008F938FE896E021C080911101681720F47B
:104F9000861B8093110102C01092110180911101B2
:104FA0001F928F9386E796E010C0809110016817DA
:104FB00020F4861B8093100102C010921001809192
:104FC00010011F928F938BE596E09F938F930E9421
:104FD000EE070F900F900F900F900895CF93C82F6A
:104FE0001F928F9320E639E03F932F930E94EE07A4
:104FF00061E070E080E090E004C0660F771F881FDA
:10500000991FCA95D2F70E949D1E0F900F900F9086
:105010000F90CF910C94A11ACF938D3109F465C0F4
:10502000B0F58E3009F4CBC100F5873009F49BC18F
:10503000A8F4863009F06AC28091D701817F8E7F03
:105040008093D70185E699E00E94550787EA9DE0A5
:105050000E94550781E08093E70180C1883009F400
:105060004FC08B3009F47CC151C2863109F4EDC1C7
:1050700038F4803109F4B6C1813109F42DC246C239
:10508000893109F4CBC18B3109F486C13FC2853324
:1050900009F434C248F4873209F430C208F430C24B
:1050A000893209F42BC232C2833438F48A3308F0CF
:1050B00029C2883309F454C129C2833409F41EC2B9
:1050C000883409F023C20E94A11A86E99DE00E945B
:1050D00055079FEF23ED80E3915020408040E1F79A
:1050E00000C000000E94382239C186EB9DE00E947A
:1050F00055070E94052C0E94DE140E941C0D2EC133
:105100008BEA9DE00E94550786E79BE00E945507C9
:105110000E94FC231F928F9383E79BE09F938F93C2
:105120000E94EE0781E79BE00E9455070E94F3234F
:10513000C82F8EE59BE00E9455071F92CF9329E56B
:105140003BE03F932F930E94EE0787E59BE00E9490
:1051500055078DE49BE00E9455078C2F81701F92AC
:105160008F932AE43BE03F932F930E94EE0788E45D
:105170009BE00E9455078EE39BE00E945507C1FB10
:10518000882780F91F928F932BE33BE03F932F9367
:105190000E94EE0789E39BE00E9455078DE29BE0A9
:1051A0000E945507C2FB882780F91F928F932AE23D
:1051B0003BE03F932F930E94EE0788E29BE00E9422
:1051C00055078FE19BE00E945507C3FBCC27C0F930
:1051D0001F92CF938CE19BE09F938F930E94EE07E9
:1051E0008AE19BE00E9455070E940524C82F86E0B3
:1051F0009BE00E9455071F92CF9321E03BE03F9335
:105200002F930E94EE078FEF9AE00E94550786EEDB
:105210009AE00E9455078C2F81701F928F9323EE86
:105220003AE03F932F930E94EE078DB79EB780968A
:105230000FB6F8949EBF0FBE8DBF81EE9AE00E941C
:1052400055078AEC9AE00E945507C1FB882780F930
:105250001F928F9327EC3AE03F932F930E94EE0723
:1052600085EC9AE00E94550783EB9AE00E9455076F
:10527000C2FB882780F91F928F9320EB3AE03F937F
:105280002F930E94EE078EEA9AE00E9455078CE960
:105290009AE00E945507C3FB882780F91F928F93DD
:1052A00029E93AE03F932F930E94EE0787E99AE0BD
:1052B0000E9455078DE89AE00E945507C4FB882795
:1052C00080F91F928F932AE83AE03F932F930E9430
:1052D000EE0788E89AE00E94550786E79AE00E9468
:1052E0005507C5FB882780F91F928F9323E73AE083
:1052F0003F932F930E94EE0781E79AE00E945507A3
:1053000085E59AE00E945507C6FB882780F91F9221
:105310008F9322E53AE03F932F930E94EE0780E5BA
:105320009AE00E94550788E49AE00E945507C7FB5F
:10533000CC27C0F91F92CF9385E49AE09F938F9377
:105340000E94EE0783E49AE00E9455078DB79EB74E
:105350004C960FB6F8949EBF0FBE8DBFC1E0DBC068
:105360008CE899E058C08091D701C82FC17080FFA8
:1053700009C089E89DE00E9455078091D701817F8F
:105380008E7F44C08DE79DE00E9455078091D70134
:1053900081608093D701E2CF8091D70181FBCC2738
:1053A000C0F991E0C927C0FB81F98093D701CC23D4
:1053B00019F080E79DE025C082E69DE02CC0809139
:1053C000D70182FBCC27C0F991E0C927C0FB82F945
:1053D0008093D701CC2319F083E59DE012C083E4CC
:1053E0009DE019C08091D70183FBCC27C0F991E0E3
:1053F000C927C0FB83F98093D701CC2351F087E301
:105400009DE00E9455078091D70181608093D7016C
:1054100082C08AE29DE00E945507A0CF8BE19DE00B
:105420000E9455078FEE9CE00E94550782EB9CE09E
:105430000E94550785E89CE00E94550781E49CE0A6
:105440000E94550786E19CE0E6CF88E09CE00E9440
:1054500055070E94DE141F928F938EEE9BE09F9360
:105460008F930E94EE0780910C011F928F9387ED1E
:105470009BE09F938F930E94EE0780916E011F9295
:105480008F9384EC9BE09F938F930E94EE07809113
:105490000D011F928F9381EB9BE09F938F930E944E
:1054A000EE078091D9019091DA01A091DB01B091D2
:1054B000DC01BF93AF939F938F938DE99BE09F9304
:1054C0008F930E94EE078DB79EB746960FB6F8945D
:1054D0009EBF0FBE8DBF42CF0E94A11AC0910D0189
:1054E00081E0C827C0930D01CC2329F083E99BE01C
:1054F0000E94550710C088E89BE08DCF80E003C074
:105500008D5101C089530E94EE2728CF86E89BE089
:105510000E945507C0E08C2FCF91089580E0089538
:1055200080E00895CF93C82F8091E701813081F00A
:1055300020F0823009F44CC042C1A0910E01B0911C
:105540000F018C91813169F0823209F03AC109C0B2
:10555000A0910E01B0910F018C91813111F0823236
:1055600049F48C2F0E948E2A81112FC08C2F0E940B
:105570000C282CC08C2F0E94902A811126C0C43187
:10558000E1F070F4CB3081F0C031D1F40E94B62646
:1055900088E599E00E94550782E08093E70115C0F5
:1055A000C93259F0C83361F485E699E00E94550785
:1055B0008CE599E00E94550708C01092E70103C1ED
:1055C00086E599E00E945507FEC081E08170FDC02C
:1055D000C43220F5CE3108F0C0C0CB3099F1C8F408
:1055E000C73009F0D2C08AE08093150194E190930E
:1055F000140193E0909313018093120188E080934B
:10560000110188E2809310018CEF97E00E9455070A
:10561000BFC0C33149F1C431C1F0B7C0CB3409F4C4
:10562000A9C028F4C93289F0C83361F0AEC0C135D1
:1056300009F49EC0C23509F499C0CE3409F0A5C062
:105640006AE09EC00E94B626A3C08091E60188232E
:1056500019F01092E6019CC089E098E00E9455077D
:1056600081E08093E701B1C083EE97E00E94550787
:1056700081ED97E00E945507809115011F928F934D
:105680008EEC97E09F938F930E94EE078CEC97E04F
:105690000E9455078AEB97E00E94550780911401FC
:1056A0001F928F9387EB97E09F938F930E94EE0753
:1056B00085EB97E00E94550786EA97E00E94550720
:1056C000809113011F928F9383EA97E09F938F93AA
:1056D0000E94EE0781EA97E00E94550780E997E073
:1056E0000E945507809112011F928F938DE897E0D9
:1056F0009F938F930E94EE078BE897E00E945507D7
:1057000086E797E00E945507809111011F928F93C1
:1057100083E797E09F938F930E94EE0781E797E0DE
:105720000E9455078AE597E00E9455078091100175
:105730001F928F9387E597E09F938F930E94EE07C8
:1057400085E597E00E9455078DB79EB748960FB63E
:10575000F8949EBF0FBE8DBF1BC0CE51EC2FF0E062
:10576000E15DFE4F80818093E60112C061E003C0DD
:1057700061E006C06AE08091E6010E94CD2608C083
:105780008091E6010E94702703C08AEF97E013C062
:105790008091E601882369F01F928F9384EF97E050
:1057A0009F938F930E94EE070F900F900F900F9092
:1057B00004C081EF97E00E94550781E006C0109277
:1057C000E70180E002C080E001CFCF910895E1E8D9
:1057D000F0E08081886080838081816080838FB7E2
:1057E000F89493E09093890090ED909388008FBF98
:1057F0000895EFE6F0E08081826080830895EFE60F
:10580000F0E080818D7F80830895EFE6F0E0808175
:1058100092E08927808308951F920F920FB60F920E
:1058200011242F933F934F935F936F937F938F93A5
:105830009F93AF93BF93EF93FF938091E801909173
:10584000E90101969093E9018093E801811103C079
:1058500082E00E941C0DE091E901E695E695F0E0FA
:10586000EA53F24FE4918091E8018E1303C080E087
:105870000E941C0DFF91EF91BF91AF919F918F916D
:105880007F916F915F914F913F912F910F900FBE3C
:105890000F901F90189504D06894B1118DC0089591
:1058A00070D088F09F5790F0B92F9927B751A0F08A
:1058B000D1F0660F771F881F991F1AF0BA95C9F7A4
:1058C00012C0B13081F077D0B1E0089574C0672F75
:1058D000782F8827B85F39F0B93FCCF38695779554
:1058E0006795B395D9F73EF490958095709561953D
:1058F0007F4F8F4F9F4F0895E89409C097FB3EF468
:1059000090958095709561957F4F8F4F9F4F99230C
:10591000A9F0F92F96E9BB279395F695879577958A
:105920006795B795F111F8CFFAF4BB0F11F460FF4A
:105930001BC06F5F7F4F8F4F9F4F16C0882311F0A2
:1059400096E911C0772321F09EE8872F762F05C0B6
:10595000662371F096E8862F70E060E02AF09A9551
:10596000660F771F881FDAF7880F9695879597F946
:10597000089557FD9058440F551F59F05F3F71F03F
:105980004795880F97FB991F61F09F3F79F08795A6
:105990000895121613061406551FF2CF4695F1DF2F
:1059A00008C0161617061806991FF1CF86957105BF
:1059B000610508940895E894BB2766277727CB01F3
:1059C00097F908950BD078C069D028F06ED018F000
:1059D000952309F05AC05FC01124EECFCADFA0F3AF
:1059E000959FD1F3950F50E0551F629FF001729F74
:1059F000BB27F00DB11D639FAA27F00DB11DAA1F93
:105A0000649F6627B00DA11D661F829F2227B00DDF
:105A1000A11D621F739FB00DA11D621F839FA00D6A
:105A2000611D221F749F3327A00D611D231F849FBA
:105A3000600D211D822F762F6A2F11249F57504011
:105A40008AF0E1F088234AF0EE0FFF1FBB1F661FAC
:105A5000771F881F91505040A9F79E3F510570F065
:105A600014C0AACF5F3FECF3983EDCF386957795A0
:105A70006795B795F795E7959F5FC1F7FE2B880F60
:105A8000911D9695879597F9089597F99F6780E8F6
:105A900070E060E008959FEF80EC089500240A9480
:105AA0001616170618060906089500240A941216F9
:105AB0001306140605060895092E0394000C11F42C
:105AC000882352F0BB0F40F4BF2B11F460FF04C0D9
:105AD0006F5F7F4F8F4F9F4F0895991B79E004C0F0
:105AE000991F961708F0961B881F7A95C9F780951D
:105AF000089597FB072E16F4009407D077FD09D080
:105B00000E94932D07FC05D03EF4909581959F4F00
:105B10000895709561957F4F0895EE0FFF1F0590D2
:105B2000F491E02D0994AA1BBB1B51E107C0AA1FE9
:105B3000BB1FA617B70710F0A61BB70B881F991F2E
:105B40005A95A9F780959095BC01CD010895F999D2
:105B5000FECF92BD81BDF89A992780B50895A8E13E
:105B6000B0E042E050E00C94CA2D262FF999FECF08
:105B70001FBA92BD81BD20BD0FB6F894FA9AF99A6A
:105B80000FBE019608950E94B52D272F0C94B62DB7
:105B9000DC01CB01FC01F999FECF06C0F2BDE1BDED
:105BA000F89A319600B40D9241505040B8F70895DC
:045BB000F894FFCF97
:105BB40020021D0D0E0EEB0DB70D840D0101C50164
:105BC40028080A03140A3F4D3620394605F904C350
:105BD40004A3046A04DD03F6030F04280448040143
:0A5BE400020304050607080900008B
:00000001FF
